:100000000C94CB040C94F3040C94F3040C94F304BC
:100010000C94F3040C94F3040C94F3040C94F30484
:100020000C94F3040C94F3040C94530F0C94C20F2F
:100030000C94F3040C94F3040C94F3040C94F30464
:100040000C94F3040C94F3040C94F3040C94F30454
:100050000C94F3040C94F3040C94F3040C945512D4
:100060000C94F3040C94F3040C94F3040C94F30434
:100070000C94F3040C94F3040C94F3040C94F30424
:100080000C94F4110C94F3040C94F3040C94F30406
:100090000C94F3040C94F3040C94F3040C94F30404
:1000A0000C94F3040C949F120C94F304A83FA80042
:1000B00000000000003E5B4F5B3E3E6B4F6B3E1C02
:1000C0003E7C3E1C183C7E3C181C577D571C1C5E19
:1000D0007F5E1C00183C1800FFE7C3E7FF001824F0
:1000E0001800FFE7DBE7FF30483A060E262979299A
:1000F00026407F050507407F05253F5A3CE73C5ACF
:100100007F3E1C1C08081C1C3E7F14227F22145FAB
:100110005F005F5F06097F017F006689956A606006
:1001200060606094A2FFA29408047E040810207E00
:10013000201008082A1C08081C2A08081E10101085
:10014000100C1E0C1E0C30383E3830060E3E0E06CB
:10015000000000000000005F00000007000700141E
:100160007F147F14242A7F2A1223130864623649DD
:100170005620500008070300001C224100004122C5
:100180001C002A1C7F1C2A08083E080800807030CA
:100190000008080808080000606000201008040239
:1001A0003E5149453E00427F40007249494946213F
:1001B00041494D331814127F1027454545393C4AB3
:1001C00049493141211109073649494936464949CA
:1001D000291E000014000000403400000008142212
:1001E0004114141414140041221408020159090680
:1001F0003E415D594E7C1211127C7F494949363E81
:10020000414141227F4141413E7F494949417F0966
:100210000909013E414151737F0808087F00417F71
:1002200041002040413F017F081422417F4040406F
:10023000407F021C027F7F0408107F3E4141413E07
:100240007F090909063E4151215E7F091929462689
:100250004949493203017F01033F4040403F1F208D
:1002600040201F3F4038403F631408146303047864
:1002700004036159494D43007F4141410204081084
:1002800020004141417F04020102044040404040BF
:10029000000307080020545478407F28444438382D
:1002A00044444428384444287F385454541800089F
:1002B0007E090218A4A49C787F0804047800447D79
:1002C00040002040403D007F1028440000417F4016
:1002D000007C047804787C0804047838444444386A
:1002E000FC1824241818242418FC7C08040408484A
:1002F0005454542404043F44243C4040207C1C209B
:1003000040201C3C4030403C44281028444C9090F5
:10031000907C4464544C440008364100000077004F
:1003200000004136080002010204023C2623263C5C
:100330001EA1A161123A4040207A385454555921E7
:1003400055557941215454784121555478402054D1
:100350005579400C1E52721239555555593954541D
:10036000545939555454580000457C410002457D8C
:10037000420001457C40F0292429F0F0282528F08E
:100380007C545545002054547C547C0A097F4932E2
:10039000494949323248484832324A4848303A415D
:1003A00041217A3A42402078009DA0A07D39444402
:1003B00044393D4040403D3C24FF2424487E49438D
:1003C000662B2FFC2F2BFF0929F620C0887E0903FE
:1003D00020545479410000447D413048484A323825
:1003E0004040227A007A0A0A727D0D19317D262951
:1003F000292F28262929292630484D402038080849
:10040000080808080808382F10C8ACBA2F1028347C
:10041000FA00007B000008142A142222142A14086F
:100420009500220095AA005500AAAA55AA55AA002F
:100430000000FF00101010FF00141414FF00101033
:10044000FF00FF1010F010F0141414FC001414F747
:1004500000FF0000FF00FF1414F404FC1414171034
:100460001F10101F101F1414141F00101010F00084
:100470000000001F101010101F10101010F01000BE
:100480000000FF101010101010101010FF100000CE
:1004900000FF140000FF00FF00001F10170000FC09
:1004A00004F414141710171414F404F40000FF00DB
:1004B000F714141414141414F700F7141414171464
:1004C00010101F101F141414F4141010F010F0006A
:1004D000001F101F0000001F14000000FC1400008B
:1004E000F010F01010FF10FF141414FF141010106F
:1004F0001F00000000F010FFFFFFFFFFF0F0F0F022
:10050000F0FFFFFF0000000000FFFF0F0F0F0F0FB5
:1005100038444438447C2A2A3E147E0202060602ED
:100520007E027E0263554941633844443C04407E68
:10053000201E2006027E020299A5E7A5991C2A49E1
:100540002A1C4C7201724C304A4D4D30304878486C
:1005500030BC625A463D3E494949007E0101017E58
:100560002A2A2A2A2A44445F444440514A444040AB
:10057000444A51400000FF0103E080FF00000808EA
:100580006B6B083612362436060F090F060000186A
:10059000180000001010003040FF0101001F010191
:1005A0001E00191D1712003C3C3C3C0000000000DE
:1005B00000B00000A170E150964F26900F1D070C6F
:1005C000009669004AE44A004844400080681000F0
:1005D0000F99FB8F9DBDBBFB77D4D4DF1F1A1AFE8A
:1005E0007F5D5DFF805A0000A0A4AA0010BA34000D
:1005F000FF5953F3FF9B9B9EFFB9B996FF9595D189
:100600009FF4940FFC295F91FF1838F8FF9294FF34
:10061000FF95D5F7BFB5DDD7F18F81F1F788C8F722
:1006200079C6467909FD9B090196F800828182808E
:10063000507162007756560076763700A2B7730184
:1006400007720600782750007334740077517600E3
:100650007F55F700477110003247720073647300D2
:1006600015A2750061679400009F6060F4F2F6F2D5
:10067000D5F08D14A1C881CFD9F1AF2000F0F89C3E
:100680008E8783878E9CF8F00000FEFF0303030330
:1006900003070EFCF80000FEFF0303030303070E2D
:1006A000FCF80000FFFF00000000000000FFFF005A
:1006B00000FEFF8383838383C7EE7C380000F8FC51
:1006C0000E07030303070EFCF800003F7FE0C08025
:1006D00080C0E07F3FFFFF01010101010101FFFF39
:1006E0000000FFFF0C0C0C0C1C3E77E3C100007FE8
:1006F000FFC0C0C0C0C0E0703F1F00001F3F70E0DF
:10070000C0C0C0E0703F1F00007FFFC1C1C1C1C1B8
:10071000E3773E1C00001F3F70E0C0C0C0E0703FA8
:100720001F000000000001FFFF01000000C0A0D971
:100730002181FFA800B801F40100000A00EE01F4D5
:1007400001000019000601FA0000000A005D01FA2C
:100750000000000A005D01FA00000019002601FAFD
:100760000000000A002601FA0000000A005D01FAFC
:100770000000000A005D01F401000019002601FAE2
:1007800000000019004A01FA0000000A004A01FABC
:100790000000000A004A01FA0000000A004A01FABB
:1007A00000000019002601FA00000019004A01FAB1
:1007B0000000000A005D01FA0000000A005D01FA75
:1007C0000000000A00AF00F40100001900AF00FAB9
:1007D00000000019005D01F40100000A00AF00F400
:1007E0000100001900C400FA0000000A00AF00FA7E
:1007F0000000000A00C400FA0000000A002601F40C
:100800000100001900A500FA0000000A00A500FA86
:100810000000000A009300FA00000019004A01FAE3
:100820000000000A002601FA0000000A000601FA92
:100830000000000A000601FA00000019005D01F442
:100840000100000A00AF00F40100001900C400FA22
:100850000000000A00AF00FA0000000A00C400FA1D
:100860000000000A002601F40100001900A500FAAA
:100870000000000A00A500FA0000000A009300FA38
:1008800000000019004A01FA0000000A002601FADF
:100890000000000A000601FA0000000A000601FA42
:1008A00000000032005D01F40100000A00AF00F416
:1008B00001000019005D01FA0000000A002601FA9B
:1008C0000000000A004A01FA0000000A004A01FA8A
:1008D0000000000A004A01FA00000019004A01FA6B
:1008E0000000000A005D01FA0000000A002601FA7B
:1008F0000000000A004A01FA0000000A004A01FA5A
:100900000001804C041900B00419001405640000B3
:10091000802003C8008403C800E803C800008008E2
:100920000B000202020000090400000102020000A4
:1009300005240010010524010101042402060524F8
:100940000600010705810310004009040100020AA6
:100950000000000705020240000007058302400076
:10096000000403090412010002EF02014041233692
:100970008000010102030141726475696E6F204CB1
:100980004C430041726475696E6F204C656F6E61F7
:1009900072646F00E81211241FBECFEFDAE0DEBFF1
:1009A000CDBF12E0A0E0B1E0ECEBFBE302C00590AC
:1009B0000D92A233B107D9F72AE0A2E3B2E001C059
:1009C0001D92A434B207E1F714E0CBECD4E004C0EC
:1009D0002197FE010E94D61DCA3CD107C9F70E948B
:1009E0000D130C94DC1D0C9400008091C805089533
:1009F000E4EEF5E0A0E0B8E000800EBC8111012C2F
:100A00001197A0FDFDCF0192B9F70DB40895FC0137
:100A10008091E305882311F13FB7F89482E0809339
:100A2000E9002091F200822F90E01816190614F4C4
:100A300081E090E0882339F0289844E64093E2056D
:100A40004091F1004083222339F02091F2002111DE
:100A500003C02BE62093E8003FBF08958FEF9FEF80
:100A600008952FB7F89483E08093E9009091E8000F
:100A7000892F807295FF04C09091F20080E4891B59
:100A80002FBF08958091DA0581110DC082E0809317
:100A9000D60584E08093D7051092D9051092D80529
:100AA00081E08093DA0586ED95E00895CF93DF939A
:100AB0001F92CDB7DEB76983DC01ED91FC91028016
:100AC000F381E02D41E050E0BE016F5F7F4F09955B
:100AD0000F90DF91CF91089583E08093E90080919A
:100AE000F200882319F08AE38093E80008950E94B9
:100AF000310590E00895CF93DF931F92CDB7DEB715
:100B0000FC018485958597FD08C02FEF3FEF358761
:100B100024870F90DF91CF910895CE0101960E9416
:100B20000705019719F4898190E0F3CF8FEF9FEFCC
:100B3000F0CF0F931F93CF93DF931F92CDB7DEB704
:100B40008C01FC018485958597FF0BC0CE01019631
:100B50000E940705019771F4898190E0F80195875B
:100B60008487F801848595850F90DF91CF911F913F
:100B70000F9108958FEF9FEFF1CFFC01848595854C
:100B800097FD0BC09FB7F89482E08093E9008091B5
:100B9000F2009FBF90E0019608959FB7F89482E01D
:100BA0008093E9008091F2009FBF90E0089540910A
:100BB000D0055091D1052091CE053091CF05421737
:100BC0005307B4F49091E8009570E1F39091E80038
:100BD00092FD19C08093F1008091D0059091D105CC
:100BE00001968F739927892B19F48EEF8093E80073
:100BF0008091D0059091D10501969093D105809375
:100C0000D00581E0089580E00895DF92EF92FF9291
:100C10000F931F93CF93DF93D82E8A01EB017B01B3
:100C2000E40EF51ECE15DF0559F0D7FE12C0FE0109
:100C300084910E94D70521968111F4CF0FEF1FEF09
:100C4000C801DF91CF911F910F91FF90EF90DF903E
:100C500008958881EECF0F931F93CF93DF931F9258
:100C6000CDB7DEB782E0898342E450E06FE179E0FE
:100C700080E80E9405060E944205DC0112960D9153
:100C80001C910115110589F0D801ED91FC910280AC
:100C9000F381E02DBE016F5F7F4FC801099597FD7D
:100CA00004C0F80100851185ECCF89810F90DF9198
:100CB000CF911F910F910895615030F02091F10074
:100CC000FC0120830196F8CF289884E68093E20502
:100CD0000895AF92BF92CF92DF92EF92FF920F935F
:100CE0001F93CF93DF936C017B018B01040F151FC2
:100CF000EB015E01AE18BF08C017D10759F069912A
:100D0000D601ED91FC910190F081E02DC60109958D
:100D1000892B79F7C501DF91CF911F910F91FF903A
:100D2000EF90DF90CF90BF90AF9008956F927F9239
:100D30008F929F92AF92BF92CF92DF92EF92FF92EB
:100D40000F931F93CF93DF934C017B01C22F102F82
:100D500098E0A92EB12C642E669466946694712C4A
:100D6000CA0187709927892B79F5D40117962D919F
:100D70003C91C7019927B9010E94AE1D269DF00143
:100D8000279DF00D369DF00D11248E0F9F1FD4016D
:100D90001596ED91FC91E80FF91F2081111112C0F9
:100DA000C095C223C083DF91CF911F910F91FF9017
:100DB000EF90DF90CF90BF90AF909F908F907F90FB
:100DC0006F900895C22BEECFD0E04770C42ED12C87
:100DD00083E0660C771C8A95E1F79E0101C0220F23
:100DE0004A95EAF7012FA301B701C4010E949606B4
:100DF000A301485F5F4FC5018C199D0902C0D595BD
:100E0000C7958A95E2F7A7CF5F926F927F928F92F4
:100E10009F92AF92BF92CF92DF92EF92FF920F9389
:100E20001F93CF93DF93EC016A30F1F48D859E859B
:100E30009C878B878C892F853889820F932F911DF2
:100E4000988B8F8781E090E0DF91CF911F910F9178
:100E5000FF90EF90DF90CF90BF90AF909F908F90DA
:100E60007F906F905F900895AB84BC84693031F4BB
:100E700029E0A20EB11CBC86AB86E4CF3DEFA316E1
:100E80003FEFB3060CF45DC08F819885A816B906B4
:100E90000CF057C0CF84D8888DEFC8168FEFD806D6
:100EA0000CF44FC089859A85C816D9060CF049C044
:100EB000603208F46FE780EE860F9FE9960F9A3153
:100EC00018F49FEFC91AD90A8C3011F08B3119F43C
:100ED0002FEFC21AD20A869534E0839FC0011124F5
:100EE0009C0120553A4F7901912C812C162F1170BD
:100EF000F701E80DF91D549011112DC0352D3F70EB
:100F0000532E3501680C791C8C81882361F001E037
:100F100089899A89892B09F000E02FE0A601B301A5
:100F2000CE010E9496060989252DA601B301CE01A6
:100F30000E9496068FEF881A980A94E08916910409
:100F4000B9F68B8990E004962B853C85820F931F20
:100F50009C878B8777CF52948FE05822D2CF2091F5
:100F60004802E0914602F0914702CF010296909329
:100F7000470280934602222319F0859194910895A7
:100F8000808191810895CF92DF92EF92FF92CF936B
:100F9000DF930E94AF07811520E8920791F48091BA
:100FA00071008D7F80937100109291004698479850
:100FB00010924502DF91CF91FF90EF90DF90CF909C
:100FC000089521E020934502813020E8920751F4F2
:100FD000809143029091440290934702809346028D
:100FE0000E94AF0797FD05C020914202222309F419
:100FF00054C020914102211150C021E020934902A8
:10100000EC01DF77209709F04BC081E080934A0222
:1010100046983FE9C32E3FE0D32EE12CF12CCAEFD6
:10102000D0E0E091420AF091430A0995811103C092
:1010300081E080934A0280914902882329F08091BF
:101040004A02882309F43FC047980E94AF070097DF
:10105000F1F19C01DE010E949F1DDC01CB0129E022
:10106000B595A795979587952A95D1F710929000F9
:101070002AE020939100D0929900C092980080932A
:101080004B0290934C02A0934D02B0934E0280917C
:1010900071008260809371008DCF10924902B0CFB1
:1010A0009E0150E040E060E472E48FE090E00E9436
:1010B0004B1D69017A0181E0C81AD108E108F108E5
:1010C00010924A02AECF4699BFCF479ABECF8FEF5C
:1010D0009FEFDC01CBCF9C01E1E7F0E090819D7FA9
:1010E000908381E080934802309347022093460228
:1010F00030934402209343020C94C3072D9A089521
:101100008FB18095807F669B88601C9B846008956A
:101110008EBD00000DB407FEFDCF08951092C805E6
:101120003E983F9808953E9A3F9A81E08093C80583
:101130000895CF93C82F0E948008982F9C2381E0A8
:101140009C1380E0CF91089580389105B8F4603405
:101150007105A0F420E191E061FD94E060FD990F3C
:1011600062FD9295687F269FD0011124A80FAC5193
:10117000BA4F8C9140FF03C0892B8C9308959095B2
:101180008923FBCF8F929F92AF92BF92CF92DF9233
:10119000EF92FF920F931F93CF93DF936D3089F0FF
:1011A000C0903D02D0903E026A30D1F410924002CD
:1011B00010923F0288E0C80ED11CD0923E02C0922D
:1011C0003D0281E090E0DF91CF911F910F91FF9060
:1011D000EF90DF90CF90BF90AF909F908F90089549
:1011E00000913F0210914002E5E06E9FE001112462
:1011F000C055DF4F4801F12CF5E0E12CFF1629F036
:10120000CE010196FE01E490EC01B12CA12C4E2DF3
:101210004170B6016A0D7B1DC4010E94A408E694CA
:10122000FFEFAF1ABF0A88E0A816B10481F7F39464
:10123000EFEF8E1A9E0AF6E0FF12DECF0A5F1F4F15
:101240001093400200933F02BCCF0DB407FEFDCFC8
:101250008EB5599A08950DB407FEFDCF8EB51EBC0C
:10126000089559980E944909862F0E944909852F9F
:101270000E944909842F0C944909462F50914F022E
:10128000570F60915002681F83E00E9431091EBC15
:1012900008958EBD00008EB50DB407FEFCCF0895F5
:1012A0003FB7F8948091390290913A02A0913B02A5
:1012B000B0913C0226B5A89B05C02F3F19F00196BE
:1012C000A11DB11D3FBFBA2FA92F982F8827BC01A0
:1012D000CD01620F711D811D911D42E0660F771FC8
:1012E000881F991F4A95D1F708958F929F92AF92C8
:1012F000BF92CF92DF92EF92FF926B017C010E942E
:1013000050094B015C01C114D104E104F104B9F0AE
:101310000E945009681979098A099B09683E73403F
:101320008105910580F381E0C81AD108E108F10830
:1013300028EE820E23E0921EA11CB11CE4CFFF9088
:10134000EF90DF90CF90BF90AF909F908F900895D7
:101350008F929F92AF92BF92CF92DF92EF92FF92C5
:101360000F931F93CF93DF936C017B018A018091D0
:101370001701882309F45CC08091E305882309F4F0
:1013800057C08091D50580FF05C08091E000826044
:101390008093E000E801B12C8AEFA82E93E0892E1B
:1013A0002AE3922E209711F4BB20D9F10E94310537
:1013B00081110AC0AA94AA20D9F161E070E080E00E
:1013C00090E00E947509EECF8C171D0611F00CF00D
:1013D0008C2F9FB7F8948092E9002091E80025FDBA
:1013E00002C09FBFDFCF282F30E0C21BD30BF70115
:1013F000815020F041914093F100FACFE20EF31EAC
:10140000BB2021F09092E800B12CEBCF8091E80056
:1014100085FDE7CF9092E800BB24B394209709F3B1
:10142000F3CF5D9884E68093D405101611063CF046
:1014300081E090E0F6019383828310E000E0C80130
:10144000DF91CF911F910F91FF90EF90DF90CF90A0
:10145000BF90AF909F908F900895BC0190E080E086
:101460000C9475096F927F928F92AF92BF92CF9238
:10147000DF92EF92FF920F931F93CF93DF93322F60
:101480003701802EC114D104A1F0369536953695DA
:10149000A0FC330F349FF001ED9D700C811CFC9D6E
:1014A000700C811CFD9D800CEC9D600C711C112446
:1014B000811C322F242FF32EA4EEB5E0FC01E82C82
:1014C00063018E2F1127822EF694F694F69491E004
:1014D00061FD94E060FD990F62FD9295CC27C09567
:1014E000DC2FA2FC05C03FEF399FE001C095D095ED
:1014F000759567957595679575956795062F0F3F57
:101500004CF40095F01AA0FC000F029FC00CD11CF7
:10151000E11E0FEFF7FF0BC08E0EA0FE02C0EE0F14
:10152000FF1FCE1ADF0AE10AF7FDE394882730E8AF
:101530000303080EA00DB11D381B831608F0832E7F
:1015400037E0301B3F1514F4F32E139530E83819AB
:10155000422F5527A1FC02C04819550BA0FE02C01E
:10156000440F551F11248F2DF82C63E0862E009018
:101570004F02D00C00905002E01C18C059988EBC4D
:10158000C40ED51EE11CBB242F1509F0B3940CD05A
:10159000EEBC07D0DEBC05D0CEBC03D01EBC03D051
:1015A0000895C8950000C895C8950895C41AD50A2D
:1015B000E108E4DF01151CF0882371F564C0A05830
:1015C000BF4F7F2CA0FC0CC06EB51EBC699F6C90F9
:1015D0006D2261286D92C89500C07A94A9F711C058
:1015E0006EB51EBC699FB001DEDFCEB51EBCC99FC3
:1015F000E0016C90D0956D22672A6D92C8957A941F
:1016000079F71124AF19B1098A9509F45CC0BB20A0
:1016100019F00DB4599AB2DFFD01E058FF4F7F2C4D
:10162000A0FC0EC06EB51EBC699F6C906C22602839
:101630006D9260806D22612861927A9499F716C04C
:101640006EB51EBC699FB0016C90D081AEDF00C04A
:10165000CEB51EBCC99F00946020662A6D9210947E
:10166000D121D72BD19300007A9451F71124A30FE5
:10167000B11D8A9561F6112331F1BB2021F00DB423
:10168000599A7CDFC895A0FC0CC06EB51EBC699F42
:101690006C906C2260286D92C89500C0FA94A9F7EE
:1016A00012C06EB51EBC699FB0017DDF8EB51EBC39
:1016B000899F802D6C9080956822662A6D92C895CE
:1016C000FA9479F7C8951124599A0DB4DF91CF9106
:1016D0001F910F91FF90EF90DF90CF90BF90AF9050
:1016E0008F907F906F9008956F927F928F92AF92BC
:1016F000CF92DF92EF92FF920F931F93CF93DF93DE
:10170000EC013A01862E6901862FBA010E943D093B
:101710000E942B09182F0E942509C034D105BCF462
:101720001123A9F09E01280F311D121613067CF417
:10173000082D730192E0E90EF11C011D92E0A92E23
:10174000282F412FBE0190E080E00E94320ADF91F5
:10175000CF911F910F91FF90EF90DF90CF90AF90BE
:101760008F907F906F90089530E73CBDDC0130E8AA
:10177000439FC0011124A80FB91F5E91352F61113D
:10178000372F3C93C89500C052235EBD0197A9F73F
:1017900004D003D030E50DB43CBD0895CF93DF9362
:1017A00010920D0410920C048091B4059091B5052F
:1017B00001969093B5058093B40548E652E0E0E1C8
:1017C000F4E0EF01DA018D91899322E0AB37B207A3
:1017D000D1F780EA95E030E020E0DC01A20FB31FF2
:1017E000ED01649768816C932F5F3F4F2331310582
:1017F000A1F7449724E08031920769F784E1DA0188
:1018000093E154962C9154972D939150D1F7815098
:101810004C5E5F4F8111F3CF83E294E01192DF01C0
:10182000A157BE4F1C928E179F07C1F7DF91CF9132
:101830000895CF93DF9310920D0410920C048091C1
:10184000B4059091B50501979093B5058093B405C3
:1018500020E134E0E8E6F2E0EF01D9018D918993CF
:1018600084E0A332B807D1F784E1D90193E154961B
:101870004C9154974D939150D1F781502C5E3F4F2E
:101880008111F3CF88EF93E030E020E0DC01A20F7C
:10189000B31FED01649748814C932F5F3F4F233175
:1018A0003105A1F7449722E08836920769F78BE764
:1018B00092E01192DF01A157BE4F1C928E179F0735
:1018C000C1F7DF91CF9108954F925F926F927F920F
:1018D0008F92AF92BF92CF92DF92EF92FF920F93CF
:1018E0001F93CF93DF93EC012B013901842E842FBA
:1018F000B9010E943D090E942B09B82E0E942509BA
:10190000C038D105FCF490E449165104DCF49E0182
:101910002B0D311D12161306ACF49201280F311D48
:10192000121613067CF492E0690E711C811C93E080
:10193000A92E6801082D7301282F4B2DB201CE016D
:101940000E94320ADF91CF911F910F91FF90EF908B
:10195000DF90CF90BF90AF908F907F906F905F900F
:101960004F9008951F93CF93DF93EC01162F5C984F
:10197000FE018591EF010E9488081150C9F75C9A19
:10198000DF91CF911F9108950F931F93CF93DF9312
:10199000F89490913302911109C093B7916093BF6D
:1019A0007894889593B79E7F93BFF2CF10923302BD
:1019B00078940091320211E0100F133088F5111164
:1019C00004C0C1E0DFEF811102C0C1E0D0E02FE729
:1019D00041E050E0BE0184E699E00E94B40B62E071
:1019E0008CEA90E00E94B20C2FEF47E051E0BE017C
:1019F00084EE95E00E94B40B62E08EEA90E00E94D3
:101A0000B20C023030F0809151028F5F809351020E
:101A100010E010933202DF91CF911F910F91089542
:101A2000882399F22FE741E050E061E07FEF84E600
:101A300099E00E94B40B62E08CEA90E00E94B20C44
:101A40002FEF47E051E061E07FEF84EE95E00E94E8
:101A5000B40B62E08EEA90E00E94B20CD4CF0895FD
:101A600090E080E008955F926F927F928F929F92B4
:101A7000AF92BF92CF92DF92EF92FF920F931F939C
:101A8000CF93DF93F12C64E1E62E7EE1C72ED12CBB
:101A9000E2E09E2EF5E08F2EA4E07A2ECF2DD0E04E
:101AA0008091B4059091B5050996C817D907BCF582
:101AB0002196EC9E8001ED9E100D1124005F1B4FBE
:101AC000F80110820E94251D5C010E94251D609175
:101AD0000001709101010E94AE1D9C01C501B6017B
:101AE0000E94AE1D029711F4F80190822430310556
:101AF00051F4EC9EF001ED9EF00D1124E859FD4FDC
:101B00007082F394CBCF25303105D9F7EC9EF001EC
:101B1000ED9EF00D1124E05FFB4F8082F2CFF12C9F
:101B200089E0C82ED12C94E1E92E2EE1A22EB12C11
:101B300032E0732E45E0642E54E0552E8091B405BA
:101B40009091B5059601281B390BCF2DD0E0C21717
:101B5000D307BCF52196EC9E8001ED9E100D11245B
:101B600008591D4FF80110820E94251D4C010E944A
:101B7000251D60910001709101010E94AE1D9C0124
:101B8000C401B5010E94AE1D029711F4F8017082E4
:101B90002430310551F4EC9EF001ED9EF00D11243E
:101BA000E859FD4F5082F394C9CF25303105D9F75C
:101BB000EC9EF001ED9EF00D1124E859FD4F60827E
:101BC000F2CF40E0099664E14817190664F4469F95
:101BD000F0011124E05FFB4F54E17181719351508A
:101BE000E1F74F5FF1CF40E064E14217130664F480
:101BF000469FF0011124E859FD4F54E17181719322
:101C00005150E1F74F5FF1CF019654E1589FF00139
:101C1000599FF00D1124E05FFB4F41E040832F5F9F
:101C20003F4F529FF001539FF00D1124E859FD4F93
:101C30004083109253021092520210920F0410929D
:101C40000E0480910001909101018A3191052CF0E0
:101C500001979093010180930001DF91CF911F9133
:101C60000F91FF90EF90DF90CF90BF90AF909F903B
:101C70008F907F906F905F900895BF92CF92DF9288
:101C8000EF92FF920F931F93CF93DF93D0E0C0E0CA
:101C900024E1C22ED12C04E132E0B32E10E00C9FDF
:101CA000C0010D9F900D11249C01205F3B4F7901D5
:101CB00080910501181768F40E94251DB6010E9445
:101CC000AE1D0A9721F4F701E10FF11DB0821F5FED
:101CD000EFCF2196C930D10509F7D0E0C0E084E10B
:101CE000C82ED12C04E192E0B92E10E00C9FC00167
:101CF0000D9F900D11249C0128593D4F7901809131
:101D00000501181768F40E94251DB6010E94AE1D3A
:101D10000A9721F4F701E10FF11DB0821F5FEFCFA9
:101D20002196C930D10509F7DF91CF911F910F910D
:101D3000FF90EF90DF90CF90BF90089581E199E000
:101D40000E946B081092CD051092B5051092B40553
:101D500010920D0410920C04109253021092520231
:101D600084E680930A018AEF90E0909301018093CA
:101D7000000187E090E090930701809306018FE0D7
:101D800090E09093090180930801109262021092F2
:101D9000CA051092B6051092CC051092CB05109290
:101DA000C60540E154E024E190E080E0FA01E80F4C
:101DB000F91F1082019684319105C1F721504C5EC4
:101DC0005F4F2111F1CF48E652E024E190E080E03E
:101DD000FA01E80FF91F1082019684319105C1F7CD
:101DE00021504C5E5F4F2111F1CF0C943D0E8F922C
:101DF0009F92AF92BF92CF92DF92EF92FF920F939A
:101E00001F93CF93DF938091620281113FC081ECD9
:101E1000E82E85E0F82E01E010E092E3A92EB12C27
:101E20002FE3922E3FE0832E45E0C42ED12CF70104
:101E300081917F01811125C00E94251DF7013197F5
:101E4000B5010E94AE1D8083E8012197FE01E9548F
:101E5000FA4F9082FE01E454FA4F80820E94251DC1
:101E6000FE01E55AFD4FB6010E94AE1D83508083EE
:101E70000E94251DCA5ADD4FB6010E94AE1D835037
:101E800088830F5F1F4F0530110589F6DF91CF91D1
:101E90001F910F91FF90EF90DF90CF90BF90AF9088
:101EA0009F908F9008951F920F920FB60F9211245A
:101EB0008F939F938091E1009091E100937F9093A5
:101EC000E10083FF0FC01092E90091E09093EB00D6
:101ED0001092EC0092E39093ED001092E30598E0ED
:101EE0009093F00082FF22C093E09093E9009091DC
:101EF000F200992319F09AE39093E8009091D405A9
:101F0000992341F09091D40591509093D40591116B
:101F100001C05D9A9091E205992341F09091E2050C
:101F200091509093E205911101C0289A84FF18C046
:101F30008091E2008E7E81608093E2008091E100DA
:101F40008F7E8093E1008091D5058E7E80618093A5
:101F5000D5059F918F910F900FBE0F901F901895F0
:101F600080FFF7CF8091E2008E7E80618093E20057
:101F70008091E1008E7E8093E1008091D5058E7E78
:101F80008160E5CF1F920F920FB60F921124CF926E
:101F9000DF92EF92FF920F931F932F933F934F93F4
:101FA0005F936F937F938F939F93AF93BF93EF93C1
:101FB000FF93CF93DF93CDB7DEB76C97DEBFCDBF76
:101FC0001092E9008091E80083FF25C068E0CE010F
:101FD00045960E945C0682EF8093E8008D8987FF1A
:101FE00039C09091E80090FFFCCF982F907609F0CF
:101FF00034C19E894F89588D2F89F88C911131C039
:10200000803861F58091D3058093F1001092F10042
:102010008EEF8093E8006C960FB6F894DEBF0FBE8B
:10202000CDBFDF91CF91FF91EF91BF91AF919F9184
:102030008F917F916F915F914F913F912F911F9160
:102040000F91FF90EF90DF90CF900F900FBE0F9009
:102050001F9018959EEF9093E800C7CF1092F10063
:10206000D5CF913059F48111D3CF4130510581F64C
:102070008091D3058D7F8093D305CACF933049F4E7
:102080008111C6CF4130510519F68091D305826088
:10209000F2CF953041F48091E80080FFFCCF2068BA
:1020A0002093E300B5CF963009F0A9C00B8D1C8DAD
:1020B00022E01092E9001092D1051092D005F212A0
:1020C0002EC01092CF051092CE050E942B061F82C3
:1020D00099E09983FA8291E09E8390EA98879AEF3B
:1020E00099872091D0053091D105275F3F4F3C83E0
:1020F0002B838D831092E9001092D1051092D005A8
:102100001093CF050093CE0549E050E0BE016F5F0C
:102110007F4F80E00E9405060E942B0679CF109326
:10212000CF050093CE050E944205DC0112960D9169
:102130001C910115110509F451C1D801ED91FC91D3
:102140000480F581E02DBE016B5E7F4FC8010995CB
:10215000009709F03EC1F80100851185EACFF3E050
:10216000FF120EC08F89882309F440C0823061F4C9
:1021700040E860E183E899E00E94B512811148CF00
:1021800081E28093EB0047CF813029F440E86BE097
:1021900087E799E0F1CF833099F70E944205DC018F
:1021A0001296ED90FC908E010F5F1F4F6801E114B5
:1021B000F10479F0D701ED91FC910680F781E02DD3
:1021C000B801C7010995080F111DF701E084F184DA
:1021D000EECFD8011C92F60101900020E9F731976B
:1021E000BF016C197D0940E0C601C6CF61E679E008
:1021F000FB01449150E080E80E94050609CF97302A
:1022000009F4BECF983021F481E08093F10000CF33
:10221000993009F0FDCE837009F0B2CFE9E1F2E028
:1022200081E031E096E32191222371F08093E9006F
:102230003093EB00DF0111972C912093EC009093E9
:10224000ED008F5F873079F78EE78093EA00109278
:10225000EA008F898093E305DBCE8B8D9C8D1092F5
:10226000E9001092D1051092D0059093CF0580938C
:10227000CE05898D811192C08E899D89913A49F44C
:10228000813209F07DCF47E050E060E171E080E00D
:10229000B3CF913209F074CF833269F48F89988D6E
:1022A000B0E0A0E080930C0190930D01A0930E018B
:1022B000B0930F01ADCE803269F48091E80082FFC7
:1022C000FCCF67E080E191E00E945C068BEF809399
:1022D000E8009ECE823209F09BCE8F898093170151
:1022E000EEEFFFE7859194918B3F9C4D51F1E0E03B
:1022F000F8E08091100190911101A0911201B0912C
:102300001301803B9440A105B105F1F480911701C0
:1023100080FD1AC0EE3F8AE0F80789F587E797E766
:1023200091838083809160008093D20588E19BE057
:102330000FB6F894A895809360000FBE909360004C
:1023400067CEEEEFFAE0D5CF80819181873797474E
:1023500009F05ECEA895809160008861809360004E
:102360008091D20580936000EE3F2AE0F20789F069
:102370008091FE0A9091FF0A9183808349CE8081EB
:1023800091818737980751F29093FF0A8093FE0A54
:10239000C5CF1092FF0A1092FE0A3ACE0E94420563
:1023A000DC0112960D911C910115110509F4E8CE7E
:1023B000D801ED91FC910190F081E02DBE016B5EA2
:1023C0007F4FC8010995811123CEF8010085118541
:1023D000EBCF181619060CF41BCED2CEF1E0FF128B
:1023E000BECE65E679E004CF1F920F920FB60F9232
:1023F00011242F933F934F935F936F937F938F930A
:102400009F93AF93BF93EF93FF9380914B02909173
:102410004C02A0914D02B0914E02892B8A2B8B2B3E
:1024200009F440C080914A0281110BC088B190E448
:10243000892788B980914902882319F088B180588A
:1024400088B980914B0290914C02A0914D02B091BD
:102450004E02181619061A061B069CF480914B02B0
:1024600090914C02A0914D02B0914E020197A109AA
:10247000B10980934B0290934C02A0934D02B0930C
:102480004E02FF91EF91BF91AF919F918F917F91FC
:102490006F915F914F913F912F910F900FBE0F90D1
:1024A0001F9018950E94C307ECCF1F920F920FB692
:1024B0000F9211242F933F938F939F93AF93BF93CA
:1024C0008091350290913602A0913702B091380286
:1024D0003091340223E0230F2D3758F50196A11DCA
:1024E000B11D209334028093350290933602A0935D
:1024F0003702B09338028091390290913A02A0914C
:102500003B02B0913C020196A11DB11D809339029E
:1025100090933A02A0933B02B0933C02BF91AF91DB
:102520009F918F913F912F910F900FBE0F901F9011
:10253000189526E8230F0296A11DB11DD2CF1F9238
:102540000F920FB60F9211248F939F9381E0809387
:10255000BF0090E99093D100809333029F918F91B7
:102560000F900FBE0F901F901895EF92FF920F9350
:102570001F93CF93DF93F82E192FE62E042F81E0BF
:10258000860F880F0E94D70583E00E94D705CF2DC4
:10259000D12FEC0EFD2EF11CCE15DF05B9F007FF93
:1025A00013C0FE0184910E94D705182F80E00E947D
:1025B000D705812321968111EFCFDF91CF911F9114
:1025C0000F91FF90EF9008958881EDCF81E0F5CFD6
:1025D000E4EEF9E01382128288EE93E0A0E0B0E02E
:1025E00084839583A683B78383E292E0918380837B
:1025F0008FEF9FEF9587848785EF94E09093430A50
:102600008093420A80E090E89093410A8093400AC8
:1026100046983E9A47983F9A0895CF93DF93CDB757
:10262000DEB7C954D1090FB6F894DEBF0FBECDBFD7
:10263000789484B5826084BD84B5816084BD85B59D
:10264000826085BD85B5816085BD80916E008160A9
:1026500080936E001092810080918100826080934F
:102660008100809181008160809381008091800051
:1026700081608093800080919100826080939100BE
:1026800080919100816080939100809190008160A1
:10269000809390008091C10084608093C1008091FC
:1026A000C10082608093C1008091C10081608093ED
:1026B000C1008091C30081608093C3008091C000FD
:1026C00082608093C0008091C20081608093C200CC
:1026D00080917A00846080937A0080917A00826091
:1026E00080937A0080917A00816080937A00809153
:1026F0007A00806880937A001092E3051092D305E7
:102700001092D5058091D70081608093D70080EA30
:102710008093D80089B5806189BD89B5826089BD03
:1027200009B400FEFDCF61E070E080E090E00E941F
:1027300075098091D8008F7C80618093D80080914A
:10274000E000807F8093E0008091E1008E7E8093A6
:10275000E1008DE08093E200559A209A81EC80930D
:102760007C0085B1806F85B984B1877E84B984B1DE
:10277000876E84B95E9A5F988AB1806D8AB9769ABD
:102780006E9881B3806F81BB899880B38D7080BB58
:1027900080E58CBD81E08DBD85E090E00E942D0A32
:1027A0005F9A85E090E00E942D0A5E985C9800E7B1
:1027B00016E0F80184910E9488080F5F1F4FF6E031
:1027C0000D371F07B1F75C9A81E880936400809110
:1027D000650081608093650080E00E94F80480E8D5
:1027E0000E949908882391F05C9885EA0E948808E5
:1027F0005C9A2E982F982D98809164008062809327
:10280000640081E083BF889513BEFCCF84E00E9402
:102810009908882309F448C02D9884E80E949908F3
:102820008823E1F00E947E0888EC90E00E942D0A47
:102830002F9882E090E00E94351D8F3F29F06FEFC6
:1028400082E090E00E943D1D84EF91E00E942D0AFD
:102850002F9A84E80E9499088111FBCF84E10E949D
:1028600099088823E1F00E947E0888EC90E00E949D
:102870002D0A2E9882E090E00E94351D882329F0D1
:1028800060E082E090E00E943D1D84EF91E00E94B4
:102890002D0A2E9A84E10E9499088111FBCF88ECC1
:1028A00090E00E942D0AB2CF0E947E0882E090E064
:1028B0000E94351D882309F4EFC00E94930881E02F
:1028C00090E00E94351D8470782E81E090E00E9497
:1028D000351D81FF14C071102E9801EF1FEF88E0A5
:1028E000A82EB12C9CE6E92EF12C80E40E949908D8
:1028F000882309F4D4C02E9A2F9A0E947E0882E37E
:1029000090E00E942D0A0E9480088111F8CF68E0B3
:102910008DE297E00E94B20C9FB7F89481E080931B
:10292000BF0020E92093D1001092C00029E020933D
:10293000C1008093C2001092C3001092BF00109299
:10294000BF001092BE00809172008460809372007C
:102950009FBF5E9AE4E1F0E084E79FEF2591359117
:10296000559145912851354909F4CA0180934F0288
:102970009093500259988BEA0E944909599A0E94F3
:102980003D0E8091CD055E98882309F423C181E036
:102990000E94C40C5E9A80915102882309F4C6C338
:1029A000815080935102809167028F5F833009F4D8
:1029B00013C1809367028091CD05882309F4E3C198
:1029C0008091C7058F5F843009F408C18093C705E3
:1029D0008091C605833639F48091CA05811103C000
:1029E00084EF8093CA050E94800840910A0183FF0A
:1029F00002C041112BC080915402909155028F303A
:102A000091052CF401969093550280935402809185
:102A10005402909155020F97C9F48091080190914A
:102A200009018630910594F00297909309018093F3
:102A30000801809106019091070101979093070189
:102A400080930601109255021092540220910801C1
:102A5000309109018091520290915302509161028C
:102A60005111BEC0442309F4F5C02F30310509F0DF
:102A7000CDC00396909353028093520280915202EC
:102A80009091530206962930310509F0C7C0909302
:102A9000530280935202DEC00E948E0810CF77202E
:102AA00029F00430110511F42E9A2F9881E00E942C
:102AB000F804980117FF04C022273327201B310B8D
:102AC00027703327C80117FD0796B3E095958795C2
:102AD000BA95E1F717FF05C00197A501421B530BFB
:102AE0009A01BC017695762F6627779567956C518C
:102AF0007A4FB0E0A0E01501221A330A8E3F5FEF53
:102B0000950709F446C048E550E0FD01EB52F94F46
:102B10004F012B01F0E84F0E511C8F3F9807C9F071
:102B2000F401E41BF50B64906701C41AD50AC60EC4
:102B3000D71EE62DF0E0022E02C0EE0FFF1F0A9412
:102B4000E2F7F8AFEFABF6016080FFA96F2AF6015C
:102B5000608221153105C9F0F401E41BF50B649086
:102B60006701C41AD50AC40CD51CE62DF0E0022C6E
:102B700002C0F595E7950A94E2F7F8AFEFABF601DE
:102B80006080FFA96F2AF60160824150510909F067
:102B9000C4CF0196A85ABF4F60587F4FA03BB105E4
:102BA00009F0ACCF80E00E94F8048FE090E00E9432
:102BB0002D0A0F5F1F4F0931110509F096CE7720BE
:102BC00011F02F9A2D9880E991E00E942D0A0E9421
:102BD0007E0895CE80E0DCCE81E0EBCE81E0F6CEC3
:102BE000442309F442CF2F30310509F03DC101964D
:102BF000909353028093520280915202909153021B
:102C00002930310509F038C1019641CF2D30310509
:102C100079F4049690935302809352028091520269
:102C20009091530207962730310509F430CF09C03F
:102C30002B30310509F022CF0596909353028093F3
:102C4000520280915202909153020896253031052C
:102C500009F41DCF80915202909153026AE070E016
:102C60000E94AE1D70930F0460930E042F30310547
:102C700029F46F30710514F00E94330D8091080122
:102C8000909109010D9741F480910E0490910F04E9
:102C90000D9714F00E94330D809108019091090165
:102CA0000B9741F480910E0490910F040B9714F050
:102CB0000E94330D8091080190910901099741F418
:102CC00080910E0490910F04099714F00E94330D27
:102CD0008091080190910901079741F480910E04B9
:102CE00090910F04079714F00E94330D8091080112
:102CF00090910901059741F480910E0490910F0481
:102D0000059714F00E94330D809160028F5F873029
:102D100009F4CDC0809360028091CB059091CC05E1
:102D2000181619066CF42091C705223049F4019752
:102D30009093CC058093CB05892B11F40E949E0EB5
:102D40008091CA05882339F081508093CA0581118A
:102D500002C00E949E0E809162028823A1F08150E1
:102D6000809362029091B6059F5F9093B6058111A2
:102D70000AC020E430E03093CC052093CB0583E0FB
:102D800099E00E946B0880910B01882369F0809183
:102D90000301909104010197909304018093030132
:102DA000892B01F510920B018091CD0581111FC077
:102DB0000E94251D80E40E94990881110E949308B9
:102DC00080E20E94990881110E948E0888E00E948A
:102DD0009908882339F085E397E00E946B0881E029
:102DE0008093CD058091CD05882309F49FC1809102
:102DF000CB059091CC05892B09F098C18091620296
:102E0000811109C180E40E949908882309F47CC0DB
:102E10008091B4059091B505893F9F4F0CF474C023
:102E200000910801109109010530110509F041C018
:102E300080910C0490910D048C3F4FEF94070CF49B
:102E400044C0019790930D0480930C040F3011053A
:102E500009F05AC080910C0490910D04823F3FEF1D
:102E600093070CF041C04EC02D30310571F401962E
:102E70009093530280935202809152029091530298
:102E80002730310509F4C0CE09C02B30310509F0D7
:102E9000B3CE0196909353028093520280915202D6
:102EA000909153022530310509F4AECED3CE81E0A6
:102EB00031CF0730110561F480910C0490910D041D
:102EC0008A3F5FEF95070CF0BCCF0E94190CBECF74
:102ED0000930110509F04AC580910C0490910D0448
:102EE000883FEFEF9E0774F0019790930D04809355
:102EF0000C040AC080910C0490910D04863FFFEFF2
:102F00009F0794F70E94190C80E20E949908882379
:102F100009F44CC08091B4059091B50508970CF068
:102F200045C0009108011091090105301105B9F45F
:102F300080910C0490910D0485309105D4F4019694
:102F400090930D0480930C040F30110579F5809156
:102F50000C0490910D048F309105CCF025C0073002
:102F6000110551F480910C0490910D048730910566
:102F700034F30E94CE0BE8CF0930110509F008C5E3
:102F800080910C0490910D04893091056CF40196A8
:102F900090930D0480930C0409C080910C049091CF
:102FA0000D048B3091059CF30E94CE0B88E00E94AB
:102FB0009908882319F180910A018823F9F091E09A
:102FC00090936102815080930A0180910801909151
:102FD00009018F30910594F420916002233071F43F
:102FE00002969093090180930801809106019091C7
:102FF0000701019690930701809306010E948008C3
:1030000083FD09C01092610280910A01843618F490
:103010008F5F80930A0141EC55E0A7EBB5E0FCEB34
:10302000EF2EF5E0FF2E81E090E0FA011191AF0163
:103030001123D1F09C0121503109B901655A7D4F0E
:103040000C91FB016081600F6C932A5A3D4FF70190
:103050006081F9012081260FF70120839A01215018
:1030600031091150F901108301961196FFEFEF1A03
:10307000FF0A85309105C9F680911204853019F454
:1030800094E69093620290916A02953019F494E666
:1030900090936202843049F4109212048091C60524
:1030A0008F5F8093C6050E94F70E8091FE038430E7
:1030B00049F41092FE038091C6058F5F8093C60588
:1030C0000E94F70E80912604843049F41092260461
:1030D0008091C6058F5F8093C6050E94F70E809190
:1030E0006A02843049F410926A028091C6058F5FAB
:1030F0008093C6050E94F70E80915602843049F4F1
:10310000109256028091C6058F5F8093C6050E947B
:10311000F70E80917E02843049F410927E028091F5
:10312000C6058F5F8093C6050E94F70E80910B0144
:10313000882309F4DBC0E0900301F09004012CE83F
:10314000E21621E0F20664F00091C90510E020EFDC
:1031500036E240E068E170E088E090E00E94640CB4
:10316000C7018D5791400F9760F40091C90510E099
:1031700020E030E040E068E170E084E190E00E940F
:10318000640CC70188579140059760F40091C90508
:1031900010E028EF3DE640E060E170E084E190E07F
:1031A0000E94640CC7018F5591404997B0F400917B
:1031B000C90510E020E030E040E068E170E084E123
:1031C00090E00E94640C5FE5E51651E0F50641F5DC
:1031D00081E199E00E946B0823C03EE0E31631E0F4
:1031E000F3060CF06AC080916702823049F4809146
:1031F0006502909166020196909366028093650243
:103200000091C90510E06091650270916602685EE8
:103210007F4F24ED37E340E084E190E00E94640CAE
:103220008091030190910401883C91050CF052C3F8
:1032300080916702823061F4809163029091640210
:103240008E3791052CF4019690936402809363026B
:10325000C0906302D09064028EE7C816D104A1F535
:1032600080910201882381F1873121F483E099E084
:103270000E946B0880910201815080930201E090CE
:10328000C905F12CC0906302D090640287012AE343
:1032900036E740E06AE070E0C601865691090E9478
:1032A000640C24E539E740E064E270E080E890E0F7
:1032B0008C199D090E94640C0DC34FE5E41641E092
:1032C000F4060CF080CF9CCFE090C905F12C87016B
:1032D00026EF3BE340E06AE070E0C60186569109C4
:1032E0000E94640C20E13FE340E0DECFE090C9059E
:1032F0008091CD05882309F416C38091CB05909168
:10330000CC05E091CA05ECAF009709F0F3C2E111DA
:1033100000C3E0900801F090090181E1F5E0EF16AB
:10332000F10429F027E0E216F10449F48FE08093DC
:1033300005018FE0E816F10499F485E00FC088E0FC
:1033400039E0E316F10451F087E04BE0E416F104B4
:1033500029F086E05DE0E516F10459F78093050158
:103360008091B4059091B5058F3F980709F4F7C097
:103370008E3FFFEF9F0709F4F7C08D3F2FEF9207B5
:1033800009F4F7C08C3F3FEF930709F4F7C08B3F78
:103390004FEF940709F4F7C05AE059AFEAE0EFABFA
:1033A0008A3F5FEF950709F4F3C0893F2FEF92073B
:1033B00009F4F3C0883F5FEF950709F4F3C081304B
:1033C000910509F4F4C08230910509F4F5C0833009
:1033D000910509F4F6C08430910509F4F7C08530F1
:1033E000910509F4F8C08630910509F4F9C08730D9
:1033F000910509F4FAC0089709F4FCC040E154E0D3
:103400005EAF4DAF512C412C712C612CC701880F40
:10341000991F8E0D9F1DFC01E455FE4F2A96FFAFAC
:10342000EEAF2A979C01245E3E4F24963FAF2EAF0D
:103430002497AC01445B5E4F26965FAF4EAF269754
:10344000FC01E458FE4F2896FFAFEEAF2897C090DE
:10345000C905D12C2090060130900701EDADFEADDD
:1034600084898130E9F42A96EEADFFAD2A97208158
:103470003181428160910E0470910F0471956195C4
:1034800071098FE390E082199309840D951DE091F5
:103490000C04F0910D0486018E0F9F1F0E94640C96
:1034A0001AAE24E1269DC001279D900D11249C0198
:1034B000205F3B4F21963FAF2EAF219767E0862ECE
:1034C000912C821893087FE3A72EB12CA218B30881
:1034D000A40CB51C3091050122963FAF22974AAD4E
:1034E000431708F08BC0842F90E02196EEADFFAD1E
:1034F0002197E80FF91F20812896EEADFFAD2897A0
:10350000223061F02696EEADFFAD2697243031F0E3
:10351000253009F52496EEADFFAD24972081318149
:103520004281E89EB001E99E700DF89E700D112455
:10353000680D791D80910E0490910F04681B790B22
:103540006350710980910C0490910D0486018A0DDD
:103550009B1D0E94640CFAADFF5FFAAFBBCFFBE08E
:10356000F9AF29E02FAB1CCF3CE039AF48E04FABBF
:1035700017CFEDE0E9AFF7E0FFAB17CF3EE039AF93
:1035800046E04FAB17CFEFE0E9AFF5E0FFAB1BCF65
:1035900020E129AF34E03FAB1ACF41E149AF53E01E
:1035A0005FAB19CFE2E1E9AFF2E0FFAB18CF29E062
:1035B00029AF3BE03FAB17CF48E049AF5CE05FABE2
:1035C00016CFE7E0E9AFFDE0FFAB15CF26E029AF6E
:1035D0003EE03FAB13CF45E049AF5FE05FAB0ECFBE
:1035E00084E089AF90E19FAB09CFE3E0E9AFF1E17F
:1035F000FFAB04CF22E029AF32E1EBCF2FEF621A0D
:10360000720A4DAD5EAD4C5E5F4F5EAF4DAF4E0C7E
:103610005F1C5FA9651608F41ACF38E6632E32E006
:10362000732E4FE3A42EB12CA218B308C701880F44
:10363000991F8E0D9F1DFC01E455FE4F2196FFAF93
:10364000EEAF21979C01245E3E4F38AF2FABAC010B
:10365000445B5E4F5BAF4AAFFC01E458FE4FFEAFE8
:10366000EDAFF30184898130B9F42196EEADFFAD61
:10367000219720813181428160910E0470910F0465
:1036800071956195710980910C0490910D048601EA
:103690008A0D9B1D0E94640C27E0822E912C8218BB
:1036A0009308512C412C2296FFAD22974F1658F5C6
:1036B000F301E40DF51D8081EDADFEAD823041F0EA
:1036C000EAADFBAD843021F08530B9F4EFA9F8AD57
:1036D00020813181428180910E0490910F04B401C8
:1036E000681B790B6350710980910C0490910D0453
:1036F00086018A0D9B1D0E94640CFFEF4F1A5F0A22
:103700008E0C9F1CD0CF2CAD2F5F2CAF34E1630EFD
:10371000711CAE18BF0849AD4213A3CFF701EE0FDD
:10372000FF1FEE0DFF1DE452FE4F208131814281CB
:103730008AE090E0821993096091B605680F792FAD
:10374000711D86018EE390E0821993090E94640C3A
:1037500001EC15E0EE24E394F12CF80181918F0146
:10376000882379F0C7010197FC01E454FA4F608186
:1037700070E089549A4FFC01808143E090E00E9400
:10378000A408FFEFEF1AFF0A25E0E216F10429F77B
:10379000860126EF35E540E070E060E090E080E0F3
:1037A0000E94640CD0900A018D2D86950CE310E0E8
:1037B000081B110917FF02C010E000E078013CE38C
:1037C000E316F10451F041E0B70184E090E00E947B
:1037D000A4084FEFE41AF40AF2CF0C33110549F0B4
:1037E00041E0B80185E090E00E94A4080F5F1F4F00
:1037F000F4CF88E00E9499088823F9F0D1101DC009
:103800008091C7058230C9F403E010E041E063E035
:1038100070E0C8010E94A40841E064E070E0C801C3
:103820000E94A40841E065E070E0C8010E94A4087D
:103830000F5F1F4F0730110549F71DA21CA280E141
:1038400092E09BA38AA384EE95E098A78FA380E8DB
:1038500090E09AA789A7E0E4F0E0FCA7EBA785E059
:103860008EAB81E08DAB81E090E09CAB8BAB1EA278
:1038700086E790E098AB8FA79EA78DA781E190E0A7
:103880009AAB89AB2091C60530E050E040E019A228
:103890008E010F5D1F4FCA01B9012AE030E040E000
:1038A00050E00E947D1D605DF80162938F0121153B
:1038B00031054105510579F7309761F001900020FD
:1038C000E9F73197AF01401B510BB801CE01829649
:1038D0000E9469068091C9058F5F833009F443C057
:1038E0008093C90580E090E0892B09F44AC80E94C2
:1038F000000047C8181619064CF42E2D30E04EEE85
:103900005EE060E0805491090E94740BFCADFF23DF
:1039100009F32E2D30E042E05FE760E090E080E0C8
:103920000E94740BD7CFF12C970142ED5BE260E06F
:1039300090E080E00E94740B87012EEB34E440E0BD
:103940006FE270E087E490E00E94640C8091C8050B
:10395000882309F4BFCF20EA35E540E060E370E05A
:103960008BE590E0A7CC1092C905BCCF0B301105B8
:1039700009F4C0CA0D30110509F068CA80910C0421
:1039800090910D04843F2FEF92070CF0ADCABACA94
:103990000B30110509F401CB0D30110509F0D4CA23
:1039A00080910C0490910D048D3091050CF4EFCAB8
:1039B000FBCA8F929F92AF92BF92CF92DF92EF920B
:1039C000FF92CF93DF93EC01688179818A819B819B
:1039D000611571058105910521F464E279ED8BE5AE
:1039E00097E02DE133EF41E050E00E944B1D49018B
:1039F0005A019B01AC01A7EAB1E40E946A1D6B0168
:103A00007C01ACEEB4EFA50194010E94781DDC01AD
:103A1000CB018C0D9D1DAE1DBF1DB7FF03C00197CF
:103A2000A109B04888839983AA83BB839F77DF91DC
:103A3000CF91FF90EF90DF90CF90BF90AF909F908D
:103A40008F9008950E94D91C089588E191E00E940A
:103A5000D91C0895B0E0A0E080931801909319015B
:103A6000A0931A01B0931B010895F999FECF92BD5E
:103A700081BDF89A992780B50895262FF999FECF30
:103A80001FBA92BD81BD20BD0FB6F894FA9AF99A7B
:103A90000FBE01960895052E97FB1EF400940E9418
:103AA000621D57FD07D00E947D1D07FC03D04EF418
:103AB0000C94621D50954095309521953F4F4F4F86
:103AC0005F4F089590958095709561957F4F8F4FCA
:103AD0009F4F08950E949F1DA59F900DB49F900D2C
:103AE000A49F800D911D11240895B7FF0C946A1DA9
:103AF0000E946A1D821B930B0895A1E21A2EAA1B35
:103B0000BB1BFD010DC0AA1FBB1FEE1FFF1FA2178D
:103B1000B307E407F50720F0A21BB30BE40BF50B8A
:103B2000661F771F881F991F1A9469F76095709513
:103B3000809590959B01AC01BD01CF010895A29F96
:103B4000B001B39FC001A39F700D811D1124911D71
:103B5000B29F700D811D1124911D089597FB072EB2
:103B600016F4009407D077FD09D00E94C21D07FC0F
:103B700005D03EF4909581959F4F0895709561957D
:103B80007F4F0895AA1BBB1B51E107C0AA1FBB1F93
:103B9000A617B70710F0A61BB70B881F991F5A95D9
:103BA000A9F780959095BC01CD010895EE0FFF1FF8
:0C3BB0000590F491E02D0994F894FFCFEB
:103BBC00FA001790011307000F006401FFFFFFFFCD
:103BCC0000E1000000000000010000000000000007
:103BDC0000000000000000000000000C530000007A
:103BEC00002C5300000000585300000000C6530086
:103BFC000000004C5400000000EA540000000000DB
:103C0C0000000000000000000000005A0C00000042
:103C1C00007A0C00000000A60C00000000140D003F
:103C2C000000009A0D00000000380E00000000009B
:103C3C000000000000920800000000B20800000024
:103C4C0000DE08000000004C0900000000D2090052
:103C5C00000000700A00000000260B0000000000AD
:103C6C0000000000000000000000005846000000AA
:103C7C0000684700000000E44800000000CC4A0047
:103C8C00000000204D00000000E04F00000000008C
:103C9C0000000000002204000000004204000000AC
:103CAC00006E0400000000DC04000000006205004F
:103CBC000000004E06000000005E0700000000003F
:103CCC0004076906300D2F0D00C180810000000033
:103CDC000000005605A80977056C05BD057B059904
:023CEC000500D1
:00000001FF
